:020000040800F2
:10000000F83E0020C9010008CF2700084926000853
:10001000CD2700083B030008B34B00080000000098
:10002000000000000000000000000000D12B0008CC
:10003000E104000800000000A92B0008D32B0008F1
:10004000E3010008E3010008E3010008E301000800
:10005000E3010008E3010008E3010008E3010008F0
:10006000E3010008E3010008E3010008E3010008E0
:100070008504000891040008E3010008E30100087A
:100080009D040008A9040008E3010008E30100083A
:10009000294B0008E3010008E3010008E301000820
:1000A000E3010008E3010008E3010008E3010008A0
:1000B000E3010008E3010008E3010008E301000890
:1000C000E3010008E3010008E3010008E301000880
:1000D000E3010008E3010008912F0008B12F000898
:1000E000E3010008E3010008E301000800F002F862
:1000F00000F05AF80AA090E8000C82448344AAF168
:100100000107DA4501D100F04FF8AFF2090EBAE865
:100110000F0013F0010F18BFFB1A43F0010318473B
:10012000E4520000045300000A444FF0000C10F8A1
:10013000013B13F0070408BF10F8014B1D1108BF65
:1001400010F8015B641E05D010F8016B641E01F805
:10015000016BF9D113F0080F1EBF10F8014BAD1C55
:100160000C1B09D16D1E58BF01F801CBFAD505E073
:1001700014F8016B01F8016B6D1EF9D59142D6D3CD
:10018000704700000023002400250026103A28BFF5
:1001900078C1FBD8520728BF30C148BF0B607047F9
:1001A0001FB51FBD10B510BD00F08DF81146FFF74B
:1001B000F7FF04F059FD00F0ABF803B4FFF7F2FFCE
:1001C00003BC00F0B3F80000094880470948004725
:1001D000FEE7FEE7FEE7FEE7FEE7FEE7FEE7FEE7F7
:1001E000FEE7FEE704480549054A064B7047000054
:1001F0004F2C0008ED000008F8270020F83E0020F2
:10020000F82E0020F82E0020B2F120030AD5C2F10A
:10021000200320FA02F001FA03F321FA02F140EA86
:100220000300704721FA03F04FF0000170474FF0D0
:1002300000020429C0F0128010F0030C00F01B80B3
:10024000CCF1040CBCF1020F18BF00F8012BA8BFC1
:1002500020F8022BA1EB0C0100F00DB85FEAC17C85
:1002600024BF00F8012B00F8012B48BF00F8012B38
:1002700070474FF0000200B5134694469646203969
:1002800022BFA0E80C50A0E80C50B1F12001BFF44F
:10029000F7AF090728BFA0E80C5048BF0CC05DF8B5
:1002A00004EB890028BF40F8042B08BF704748BF03
:1002B00020F8022B11F0804F18BF00F8012B704777
:1002C000704770477047754600F02CF8AE46050041
:1002D0006946534620F00700854618B020B5FFF761
:1002E00081FFBDE820404FF000064FF000074FF0BF
:1002F00000084FF0000B21F00701AC46ACE8C00944
:10030000ACE8C009ACE8C009ACE8C0098D4670474C
:1003100010B50446AFF300802046BDE81040FFF75B
:100320004CBF000000487047982700200149182062
:10033000ABBEFEE7260002007047FEE704284FF040
:10034000000070470020704710B50022044905489E
:1003500002F048FF0449034802F03EFF002010BDB0
:1003600060210020A4130020601D002070B5054608
:100370000E460B4801210180316841602946094839
:1003800002F02AFF074802F006FF002403E0285D80
:1003900004F01AFE641C3068A042F8D8002070BD3A
:1003A0008C000020A413002010B50A460849D1F89B
:1003B000B812D1F81412002901D0012010BD014655
:1003C000034802F00FFFBDE81040014802F084BF6F
:1003D000A413002070B50024224802F0FFFF224839
:1003E00002F0DCF8214802F0D9F84FF6FF752946F3
:1003F0001F4800F037FC29461E4800F033FC294610
:100400001D4800F02FFC29461C4800F02BFC1C481E
:10041000816921F004018161816921F00801816114
:10042000816921F010018161816921F020018161E0
:10043000012080F3108801F09FFC4FF0E0210020A4
:10044000086148618861411EA00000F1E020C0F809
:100450008011C0F88012641C082CF5D3002080F3B2
:10046000108870BDA4130020041200204C1200203C
:1004700000080140000C0140001001400014014040
:1004800000100240014800F035BA0000601300205F
:10049000014800F02FBA00001C130020014800F0B2
:1004A00029BA000094120020014800F023BA00008D
:1004B000D812002030B590F840500124AC40C56BF4
:1004C0006C60046863604368102B04D00368996013
:1004D0000068C26030BD03689A600068C16030BDCA
:1004E000704772B6FEE700B585B000220192029215
:1004F00000920390049172B6694601A800F0FAFADE
:1005000020B162B64FF0FF3005B000BD62B60020EA
:10051000FAE7000006490020C8610648016941F079
:1005200004010161016941F040010161704700006F
:100530007827002000200240064A0021D1610649A8
:100540000A6942F002020A614861086940F040000D
:10055000086170477827002000200240044B0022E9
:10056000DA61044A136943F00103136101807047A3
:1005700078270020002002400088704710B504460C
:10058000D00702D04FF0FF3010BD002307E004EB8E
:100590004300FFF7F1FF41F823005B1C9BB2B3EB74
:1005A000520FF4D3002010BD00201449CA68D306AE
:1005B000134A04D5D06940F00200D0611020CB6806
:1005C0005B0705D5D36943F00103D36140F0040014
:1005D000CB69DB0707D0D36943F00403D361CA6951
:1005E00022F00102CA61A0F58072013A01D0C86010
:1005F0007047C86920F00100C861704700200240C0
:100600007827002070B5044600F0A2FC0546114E84
:1006100009E0601C07D024B100F09AFC401BA04206
:1006200001D9032070BDF068C007F2D1F0688006E0
:1006300001D52020F060F068C00605D4F069C0073D
:1006400002D1F068400703D5FFF7AEFF012070BD6F
:10065000002070BD002002402DE9F04105460F4604
:1006600016464FF000644FF0FF38A54203D31A49F5
:10067000A819884202D34046BDE8F081F00701D0B6
:100680004046F9E700F0DAFAA5F10060800A04EBD1
:1006900080200121FFF727FF18B100F07FFA4046C4
:1006A000EAE7002410E072B657F8242005EB440175
:1006B0000023012000F07CFA20B162B600F06EFA4F
:1006C0004046D9E7641CA4B2B4EB560FEBD362B634
:1006D00000F064FA0020CFE7000002082DE9F7439C
:1006E0000D46164600F0AAFA00244FF0FF38164FC8
:1006F0001DE072B635F8142000230120009900F0A7
:1007000057FA28B162B600F049FA4046BDE8FE83C8
:1007100062B6009835F814100088884203D000F0C3
:100720003DFA4046F2E70098801C0090641CB442F9
:1007300002D20098B842DCD962B600F02FFA034921
:10074000009808600020E1E7FDFF01080C00002090
:1007500070B5FF23FF22084D05F5807605E010F8FF
:10076000014B54402A5D5A40335D491E89B2F6D28E
:1007700042EA032070BD00000452000810B50B4887
:100780000168001D0468001D0068084400280BD0A3
:100790000822074901F059FF054920460422BDE817
:1007A0001040103101F051BF10BD0000E8F7FF1FED
:1007B0006E00002010B590F821100022022905D00B
:1007C0000421816380F82020012010BD01680B689E
:1007D00023F00E030B6001680B6823F001030B602C
:1007E00090F84030C46B012101FA03F3636080F894
:1007F000211080F82020104610BD000010B5002404
:1008000090F82110022903D00421816301243DE0E6
:1008100001680A6822F00E020A6001680A6822F084
:1008200001020A601A4A0168914201D1012121E0C6
:10083000174A1432914201D110211BE0144A283288
:10084000914201D1891515E0114A3C32914201D102
:1008500089140FE00E4A5032914202D14FF4803198
:1008600008E00B4A6432914202D14FF4801101E05A
:100870004FF08071064A083A5160012180F821103A
:10088000002180F82010416B01B18847204610BD3F
:100890000800024010B5002825D001680A6822F03F
:1008A00001020A600268002111600268516002685A
:1008B00091600268D1600D4B02681A441423B2FBA8
:1008C000F3F2920002640A4BC363012494405C601B
:1008D0008162C16201634163816380F8211080F805
:1008E0002010002010BD012010BD0000F8FFFDBF4A
:1008F000000002402DE9F05FC16B0A6801680B68D7
:10090000046C4FF0040A0AFA04FA4E4D4E4E4F4F53
:10091000DFF83CC1DFF83C81DFF83C911AEA020FB6
:1009200031D05FEA437A2ED50A68920603D40A686A
:1009300022F004020A600168A94201D1042119E0F1
:10094000B14201D1402115E0B94202D14FF480619A
:1009500010E0614502D14FF480410BE0414502D1E6
:100960004FF4802106E0494502D14FF4800101E0B7
:100970004FF08061334A083A5160C16A00295FD064
:10098000BDE8F05F08474FF0020E0EFA04FE1EEAC3
:10099000020F4FF0000A4FF0010B35D05FEA837E63
:1009A00032D50A68920605D40A6822F00A020A6063
:1009B00080F821B00168A94201D1022119E0B142B9
:1009C00001D1202115E0B94202D14FF4007110E0AD
:1009D000614502D14FF400510BE0414502D14FF483
:1009E000003106E0494502D14FF4001101E04FF01B
:1009F0000071144A083A516080F820A0816A0029E9
:100A00001ED0BDE8F05F08470825A540154217D065
:100A10001A0715D50A6822F00E020A6090F84010F5
:100A2000C26B0BFA01F15160C0F838B080F821B008
:100A300080F820A0016B002902D0BDE8F05F0847D4
:100A4000BDE8F09F080002401C0002403000024058
:100A500044000240580002406C00024070B5044659
:100A6000002594F8200001280CD0012084F82000F3
:100A700094F821600020012E06D084F82000022581
:100A8000284670BD022070BD022684F82160A06354
:100A90002068066826F0010606602046FFF70AFD7A
:100AA000E06A28B12068016841F00E01016009E0A8
:100AB0002068016821F0040101602068016841F0AC
:100AC0000A0101602068016841F001010160D7E777
:100AD00070B5044600F03CFA0546601C02D004489C
:100AE0000078044400F034FA401BA042FAD370BDF1
:100AF000D80000202DE9F04705460F464FF0010AC7
:100B0000DFF8908098F8180001280DD0012088F8AF
:100B100018002868204E4CF25039022807D0484669
:100B2000FFF770FD98B12FE00220BDE8F08748463E
:100B3000FFF768FDF8B90120FFF7ECFC4846FFF726
:100B400061FD8246306920F0040030611CE04FF006
:100B5000FF303860AC6811E02046FFF7EDFC4846F6
:100B6000FFF750FD8246306920F0020030615FEAF5
:100B70000A0001D03C6007E004F58064D5E9020179
:100B800000EB8120A042E7D8002088F818005046EA
:100B9000CBE70000782700200020024003480169CD
:100BA00041F08001016100207047000000200240F8
:100BB0002DE9F05F0746884615461E460024DFF8FB
:100BC000749099F81800012809D0012089F81800BC
:100BD0004CF2503B5846FFF715FD18B126E00220B5
:100BE000BDE8F09F012F05D0022F05D00427DFF8C4
:100BF00048A019E00127FAE70227F8E72201284672
:100C00003146FFF701FB81B208EB4400FFF7A6FC79
:100C10005846FFF7F7FCDAF8101021F00101CAF886
:100C2000101018B9641CE4B2BC42E7D3002189F863
:100C30001810D5E778270020002002400020064940
:100C40000A69120607D5054A4A60054A4A600969D9
:100C5000090600D5012070470020024023016745A6
:100C6000AB89EFCD2DE9F0430022DFF8CC804FF0C7
:100C70000F0C5BE0012393400B40D3B322F003043D
:100C800004EB0805AC689607370F0CFA07F606EA7E
:100C900004092A4CA04201D100240FE0284CA042B4
:100CA00001D101240AE0274CA04201D1022405E031
:100CB000254CA04201D1032400E00424BC404C4553
:100CC00013D1224C27689F432760241D27689F4328
:100CD00027601E4C0C3427689F432760241F276819
:100CE0009F432760AC68B443AC60FF2B02D8044636
:100CF00002E019E000F1040402D84FEA820503E0A3
:100D0000A2F108054FEA850526680CFA05F726EAE0
:100D100007064FF0040707FA05F746EA07062660BC
:100D2000C46824EA0304C46002F1010231FA02F348
:100D3000A0D1BDE8F08300000000014000080140A0
:100D4000000C01400010014000140140000401406B
:100D50002DE9F84F00240023DFF8C4914FF00F086D
:100D6000A9F1040B09F1040AABF1040ED1E001274B
:100D7000A7403A40BA4275D1DFF8A8C14D68A5EB4B
:100D80000C0665452BD00DDC032D34D005DC35B3C6
:100D9000012D19D0022D2FD11BE0112D16D0122DAF
:100DA0002AD119E0B6F5881F19D006DCB6F5803FC8
:100DB00015D0B6F5801F1FD111E0B6F5001F0ED07B
:100DC000B6F5041F18D10AE0CB6815E0CB681B1DEF
:100DD00012E0CB6808330FE0CB680C330CE08B6873
:100DE00023B1012B04D00823476105E0042303E06D
:100DF0000823076100E00023FF2A01D8054601E02F
:100E000000F1040502D84FEA840603E0A4F10806C5
:100E10004FEA86062F6808FA06FC27EA0C0703FA51
:100E200006F647EA06072F604D68ED0070D53E4D87
:100E3000AE6946F00106AE61AD6905F001050095A9
:100E40003A4D24F003067719BE68A5072D0F08FA5E
:100E500005FC26EA0C06DFF8D8C0604503D14FF048
:100E6000000C17E054E0DFF8CCC0604502D14FF031
:100E7000010C0FE0DFF8C0C0604502D14FF0020C5A
:100E800008E0DFF8B8C0604502D14FF0030C01E084
:100E90004FF0040C0CFA05FC4CEA060CC7F808C02D
:100EA0004D68ED0205D5D9F800501543C9F800503A
:100EB00004E0D9F800509543C9F800504D68AD02E0
:100EC00005D5DAF800501543CAF8005004E0DAF806
:100ED00000509543CAF800504D68AD0305D5DBF8C6
:100EE00000501543CBF8005004E0DBF80050954368
:100EF000CBF800504D68ED0305D5DEF800501543E2
:100F0000CEF8005004E0DEF800509543CEF80050D3
:100F1000641C0A6832FA04F57FF429AFBDE8F88F43
:100F200008040140000011100010024000000140C0
:100F300000080140000C0140001001400014014075
:100F4000002A01D001617047090401617047000067
:100F50000148806870470000D8000020024881687E
:100F60000278114481607047D800002010B507480E
:100F7000016841F010010160032000F087F80F20A4
:100F800000F006F800F026F8002010BD0020024016
:100F900070B504460D4D4FF47A712878B1FBF0F02E
:100FA0000B490968B1FBF0F001F040F908B10120EC
:100FB00070BD102C07D200222146501E00F046F8CA
:100FC0006C60002070BD012070BD0000D8000020C2
:100FD000E400002008B50C48816941F001018161FD
:100FE000816901F001010091C16941F08051C16145
:100FF000C06900F0805000900449486820F0E0602B
:1010000040F00070486008BD001002400000014040
:1010100000280DDB00F01F020121914040098000F3
:1010200000F1E020C0F88011BFF34F8FBFF36F8F46
:101030007047002809DB00F01F02012191404009A0
:10104000800000F1E020C0F800117047F0B40D46B8
:101050000D4B1B68C3F30223C3F10704042C00D912
:101060000424191D072901D2002300E0DB1E0126FC
:1010700006FA04F1491E294099409E40761E16400A
:101080003143F0BC03F096BD0CED00E000F0070129
:10109000054A10684FF6FF03184040EA0120034953
:1010A00008431060704700000CED00E00000FA05F6
:1010B000BFF34F8F05480168054A01F4E061114311
:1010C0000160BFF34F8F00BFFDE700000CED00E0B3
:1010D0000400FA0510B50C0607D501F0070101EB75
:1010E000810100EBC100103005E001EB810100EB54
:1010F000C10000F5A87099B232B1012202730181DA
:10110000190C4181002010BD00220273C180F9E753
:10111000704701EB810200EBC202D0F8D402526AA0
:1011200002F05DBB01EB810200EBC202D0F8D402F9
:10113000D2F8642102F0BEBB10B50446002C08D0E2
:10114000032084F89102206803F016FD18B10120F5
:1011500010BD012010BD204600F034FC002084F8B2
:10116000910210BD70B504460B0601F0070000EBBC
:10117000800104EBC1014FF001024FF0000502D5E0
:1011800010314A7002E001F5A8714D70087094F8B2
:101190009002012808D084F89022206803F0BEF85D
:1011A00084F89052002070BD022070BD70B50446D6
:1011B00001F00F002279904201D9012070BD0B0689
:1011C00001F0070000EB800104EBC1014FF00102C8
:1011D0004FF0000502D510314A7002E001F5A87108
:1011E0004D708D70087094F89002012808D084F832
:1011F0009022206803F044F984F89052002070BDDA
:10120000022070BD2DE9F05F0B788D6904685FEAFC
:10121000424A4FF0000C4BF68F7948F2800848F6AE
:101220008F7648F2C0074FF4806E32D5B4F850A0E4
:101230004FF0020B0BEBC30BDA440EEB4A0A34F807
:101240000A40C4F30904A54202D32D1B8D6101E0BD
:10125000C1F818C08D6955B9056835F823C00CEA86
:10126000090C8CF4005C4CEA080C25F823C05206EB
:1012700007D50B78026832F8235035403D4322F8F9
:101280002350C4B30A8949690068234603F055FC1A
:1012900031E0B4F850A04FF0060B0BEBC30BDA446F
:1012A0000EEB4A0A34F80A40C4F30904A54202D3FB
:1012B0002D1B8D6101E0C1F818C08D6955B9056815
:1012C00035F823C00CEA090C8CF4005C4CEA080CDD
:1012D00025F823C0520607D40B78026832F8235051
:1012E00035403D4322F823502CB14A8949690068B2
:1012F000234603F022FC2046BDE8F09F2DE9F05F75
:1013000005460C4616462178A36928685FEA466AB6
:1013100048F68F774CF280084FF4806E4FF0020948
:101320004FF0060C4FF0000272D5B0F850B009EB48
:10133000C10AD3440EEB4B0B30F80B00C0F309008D
:10134000834202D91B1AA36100E0A261A36973B1B1
:10135000730407D52B6833F821603E4046EA08063F
:1013600023F8216094F82410012952D07EE160789E
:1013700010B1012811D018E02868B0F850100844C6
:1013800000EB4A0000F580600188C1F3090101808B
:10139000018841F40041018007E02868B0F850104E
:1013A000084400EB4A00A0F800242868617811B1D5
:1013B000012913D01CE0B0F85010084421780CEB40
:1013C000C10100EB410000F580600188C1F3090113
:1013D0000180018841F40041018009E0B0F850101B
:1013E000084421780CEBC10100EB4100A0F8002477
:1013F00021782846FFF78DFE7004B7D5217828683C
:1014000030F821203A4042EA080220F821202DE15C
:101410005BE0616901446161E1690144E161236963
:10142000216A994203D31846091A216204E041B1A6
:1014300084F8242008462262617829B1012932D03B
:101440003CE084F82420F7E72968B1F850201144E3
:10145000227809EBC20201EB420101F580610A88A2
:10146000C2F309020A803E280BD94209C30600D103
:10147000521E0B884FF4004646EA822213430B802B
:101480001CE058B14208C30700D0521C0B884FF62D
:10149000FF7606EA822213430B800FE00A8842F4AB
:1014A00000420A800AE02968B1F8502011442278ED
:1014B00009EBC20201EB4201A1F8000483B22289C8
:1014C0006169286803F061FBD0E0B0F850A00CEB34
:1014D000C10BDA440EEB4A0A30F80A00C0F30900E7
:1014E000834202D31B1AA36100E0A261A36973B116
:1014F000730407D42B6833F821603E4046EA08069F
:1015000023F8216094F82410012955D0AEE06078CA
:1015100010B1012813D01CE02868B0F850301844EE
:1015200009EBC10100EB410000F580600188C1F3C7
:1015300009010180018841F40041018009E0286827
:10154000B0F85030184409EBC10100EB4100A0F89D
:1015500000242868617811B1012913D01CE0B0F88B
:101560005010084421780CEBC10100EB410000F55C
:1015700080600188C1F309010180018841F40041C4
:10158000018009E0B0F85010084421780CEBC1014B
:1015900000EB4100A0F8002421782846FFF7B9FDB0
:1015A000700463D42178286830F821203A4042EA58
:1015B000080220F8212059E0616901446161E16974
:1015C0000144E1612369216A994203D31846091A4B
:1015D000216204E049B10846226284F82420296887
:1015E00062782AB1012A31D03AE084F82420F6E763
:1015F000B1F85020114422780CEBC20201EB4201F9
:1016000001F580610A88C2F309020A803E280BD9DD
:101610004209C30600D1521E0B884FF4004646EA29
:10162000822213430B801BE058B14208C30700D04D
:10163000521C0B884FF6FF7606EA822213430B807A
:101640000EE00A8842F400420A8009E0B1F8502016
:10165000114422780CEBC20201EB4201A1F8000414
:1016600083B262896169286803F08FFA217828685B
:1016700030F8212048F6BF731A4082F0100282F041
:10168000200248F280031A4320F821200020BDE800
:10169000F09F01F0070101EB810100EBC100D0F8E0
:1016A0006C0170472DE9F04104460F0601F0070078
:1016B00000EB800104EBC1014FF001064FF0000583
:1016C00002D510314E7002E001F5A8714D7008701E
:1016D0000A61CB70022B00D10D7194F890020128A1
:1016E00009D084F89062206802F066FC284684F8ED
:1016F0009052BDE8F0810220FBE710B501F007042D
:1017000004EB840100EBC10101F5A8714A618B6112
:101710000022CA614A700C70006802F011FF0020BC
:1017200010BD70B504460D46217905F007008842CA
:1017300001D9012070BD29064FF000064FF00102CB
:1017400006D500EB800104EBC10110314A7006E0C0
:1017500005EB850104EBC10101F5A8714E708A709B
:10176000087094F89002012807D084F8902220682D
:1017700002F0C8FE680702D006E0022070BD04F542
:101780002671206802F07AFE84F89062002070BD15
:1017900010B501F0070404EB840100EBC101103126
:1017A0004A618B61012281F824200B620023CB6106
:1017B0004A700C70006802F0C3FE002010BD1FB517
:1017C0000446206803F0B6F9010405D504B02046AC
:1017D000BDE8104000F0FCBF41050FD5206830F88F
:1017E000441F21F480610180204600F01BF904B001
:1017F0002046BDE81040002100F02FB9410406D575
:10180000206830F8441F21F4804101801FBD81040D
:1018100006D5206830F8441F21F4005101801FBD17
:10182000C10415D5206830F8401F21F00401018063
:10183000206830F8401F21F008010180204600F0A8
:1018400004F9206830F8441F21F4805101801FBD45
:1018500001053FD5002021686A4631F8203022F882
:101860001030401CC0B20828F7D331F8400F40F0C8
:1018700001000880206830F8401F21F0010101803C
:101880002068B0F844104905FBD530F8441F21F416
:10189000806101800020236832F8101023F82010A6
:1018A000401CC0B20828F6D3206830F8401F41F031
:1018B00008010180206830F8441F21F40061018094
:1018C000206830F8401F41F004010180204600F0FC
:1018D00011F91FBD810509D5206830F8441F21F496
:1018E00000710180204600F0B4F81FBDC005FCD592
:1018F000206830F8441F21F4807101801FBD2DE95C
:10190000F0410446002C04D094F89102002518B14F
:1019100007E00120BDE8F08184F89052204600F0F5
:1019200063F8032084F891026571206802F09FFD3E
:1019300094E80F0002F0B5FC022618B184F8916219
:101940000120E7E70021206803F00DF918B184F8C1
:1019500091620120DEE7002101270BE001EB81000D
:1019600004EBC00047740174C5740562456285626A
:10197000491CC9B220798842F0D800210DE001EB62
:10198000810004EBC00000F5A87045700170C570BF
:10199000056145618561491CC9B220798842EED84C
:1019A00094E80F0002F05AFD18B184F8916201200A
:1019B000B0E7657384F89172206802F04DFD002055
:1019C000A8E7000000680649884207D10548C169B8
:1019D00021F40001C1611420FFF71ABB7047000019
:1019E000005C00400010024008B500680B498842C6
:1019F00012D10B48C16941F40001C161C06900F412
:101A000000000090002211461420FFF71FFBBDE8E4
:101A100008401420FFF70DBB08BD0000005C00402B
:101A20000010024070B504460125A079022801D0BB
:101A3000FEF757FD2946D4F8D40202F02CF8D4F86A
:101A4000D402BDE8704001F0E7BFD0F8D40202F044
:101A50000CB8D0F8D40202F012B810B5044694F8CD
:101A6000900201280AD0012084F890026173206856
:101A700003F07BF8002084F8900210BD022010BD16
:101A8000D0F8D42200F52671104602F010B810B537
:101A9000044694F89002012810D0012084F89002A6
:101AA000206803F038F801212046FFF731FB206859
:101AB00002F0D0FC002084F8900210BD022010BD7E
:101AC00010B5044694F89002012810D0012084F843
:101AD0009002206802F0CBFC00212046FFF718FBA3
:101AE000206802F0B9FC002084F8900210BD0220AA
:101AF00010BD000010B50446D4F8D40202F01FF85F
:101B0000A07A002804D00348016841F00601016072
:101B100010BD000010ED00E02DE9F8430446DFF8A9
:101B2000F8802078C0075FD00027D8F81C00C000DC
:101B30000BD4D8F81C0040F08050C8F81C00D8F82E
:101B40001C0000F0805000900127344D2868C0052B
:101B500012D4286840F480702860FFF7F9F906462F
:101B600007E0FFF7F5F9801B642802D90320BDE8E0
:101B7000F8832868C005F4D5D8F8200000F4407038
:101B800010B3A18801F4407181421DD0D8F8200023
:101B900020F44070224901220A6000220A60C8F83D
:101BA0002000C00710D0FFF7D3F9054641F2883670
:101BB00006E0FFF7CDF9401BB04201D90320D6E77C
:101BC000D8F820008007F4D5D8F82000616820F408
:101BD00040700843C8F82000012F05D1D8F81C0038
:101BE00020F08050C8F81C002078800707D5D8F86E
:101BF0000400A16820F440400843C8F8040020789D
:101C0000C00607D5D8F80400E16820F48000084336
:101C1000C8F804000020AAE700100240007000404D
:101C2000400442422DE9F04704460D46002C17D0EF
:101C3000DFF83081D8F8000000F00700A84211D288
:101C4000D8F8000020F007002843C8F80000D8F8B2
:101C5000000000F00700A84204D00120BDE8F08792
:101C60000120FBE72068404E810712D5400703D5CD
:101C7000706840F4E06070602078000703D57068F9
:101C800040F4605070607068A16820F0F000084374
:101C900070602078C0072CD06068012806D0022828
:101CA00009D0316889070BD40120D7E7316889034F
:101CB00006D40120D2E73168890101D40120CDE7A3
:101CC000716821F0030101437160FFF741F9074694
:101CD00041F2883906E0FFF73BF9C01B484501D9BE
:101CE0000320BBE77068616800F00C00B0EB810F67
:101CF000F1D1D8F8000000F00700A8420ED9D8F8BA
:101D0000000020F007002843C8F80000D8F80000C1
:101D100000F00700A84201D001209FE7207840078B
:101D200005D57068E16820F4E060084370602078B1
:101D3000000706D57068216920F4605040EAC100B0
:101D4000706000F08BF87168084AC1F30311515CB0
:101D5000C8400749086007480068FFF719F90020E4
:101D60007CE700000020024000100240F45100080F
:101D7000E4000020DC0000202DE9F041FFF7E8F846
:101D80000546324C206840F00100206007E0FFF774
:101D9000DFF8401B022802D90320BDE8F08120684B
:101DA0008007F4D5206820F0F80040F08000206023
:101DB000FFF7CEF805460027676041F2883606E057
:101DC000FFF7C6F8401BB04201D90320E5E7606881
:101DD00010F00C0FF4D11F491D4808601E48006820
:101DE000FFF7D6F808B10120D7E7FFF7B1F80546AD
:101DF000206820F08070206006E0FFF7A9F8401B03
:101E0000022801D90320C8E720688001F5D4676063
:101E1000FFF79EF80546206820F41020206006E0B9
:101E2000FFF796F8401B642801D90320B5E7206826
:101E30008003F5D4206820F480202060606A40F0A0
:101E400080706062A7600020A7E7000000100240D9
:101E500000127A00E4000020DC0000200E4B5968DC
:101E60000E4801F00C02042A11D0082A0FD10C48A8
:101E7000C1F38342805CC9030AD55968084AC1F39B
:101E80004041921E515C054A5043B0FBF1F070474F
:101E900004494843704700000010024000127A00D5
:101EA000E451000800093D002DE9F84F0446002CDC
:101EB0000ED02078D94DC0075ED06868C0F381008D
:101EC00001280BD06868C0F38100022803D00CE021
:101ED0000120BDE8F88F6868C00306D52868800334
:101EE0004AD56068A8BB0120F3E76068B0F5803F81
:101EF00011D0A8B1B0F5A02F1BD0286820F48030F5
:101F00002860286820F480202860606830B3FFF7DC
:101F10001FF806461EE0286840F480302860F4E789
:101F2000286820F480302860286820F48020286009
:101F3000EBE7286840F480202860286840F480306F
:101F40002860E2E7FFF704F8801B642802D9032029
:101F5000BFE711E028688003F4D50DE0FEF7F8FF35
:101F6000064606E0FEF7F4FF801B642801D9032033
:101F7000AFE728688003F5D42078DFF8A4828007D3
:101F80004FF0010A4FF0000945D5686810F00C0FBA
:101F900007D06868C0F38100022812D16868C003C6
:101FA0000FD42868800704D52069012801D00120BA
:101FB0008FE72868616920F0F80040EAC1002860D6
:101FC00029E02069B8B1C8F800A0FEF7C1FF0646B5
:101FD00006E0FEF7BDFF801B022801D9032078E749
:101FE00028688007F5D52868616920F0F80040EA84
:101FF000C10028600FE0C8F80090FEF7A9FF064670
:1020000006E0FEF7A5FF801B022801D9032060E748
:1020100028688007F5D42078000726D58148A16973
:1020200099B1C0F800A0FEF793FF064606E0FEF760
:102030008FFF801B022801D903204AE7686A8007C6
:10204000F5D5012000F0B2FD0FE0C0F80090FEF7DA
:102050007FFF064606E0FEF77BFF801B022801D9C2
:10206000032036E7686A8007F5D42078400773D5E7
:102070000026E869C00008D4E86940F08050E861B3
:10208000E86900F0805000900126DFF89CB1DBF891
:102090000000C00514D4DBF8000040F48070CBF8D9
:1020A0000000FEF755FF074606E0FEF751FFC01B94
:1020B000642801D903200CE7DBF80000C005F4D543
:1020C000E068012812D0B0B105281DD0286A20F0A0
:1020D00001002862286A20F004002862E06841F2CA
:1020E000883B28B3FEF734FF07461DE0286A40F01E
:1020F00001002862F2E7286A20F001002862286ABD
:1021000020F004002862E9E7286A40F00400286211
:10211000286A40F001002862E0E7FEF719FFC01BC3
:10212000584501D90320D4E6286A8007F5D50DE08B
:10213000FEF70EFF074606E0FEF70AFFC01B5845F4
:1021400001D90320C5E6286A8007F5D4012E03D102
:10215000E86920F08050E861E069A0B36968C1F3E4
:102160008101022946D0022805D0C8F86090FEF708
:10217000EFFE04463AE0C8F86090FEF7E9FE064636
:1021800006E0FEF7E5FE801B022801D90320A0E649
:1021900028688001F5D4206AB0F5803F05D16868D1
:1021A000A16820F4003008436860D4E908010843BE
:1021B000696821F4741108436860C8F860A0FEF7EC
:1021C000C7FE044607E026E0FEF7C2FE001B022819
:1021D00001D903207DE628688001F5D51BE0FEF7D4
:1021E000B7FE001B022801D9032072E6286880018F
:1021F000F5D410E001280CD06868226A00F4803120
:10220000914204D1616A00F47010884203D0012029
:102210005FE601205DE600205BE600000010024062
:1022200000004242800442420070004010B5401E4F
:10223000B0F1807F01D3012010BD4FF0E024606138
:102240000F21601702F0B6FC0020A061072020617A
:10225000002010BD38B5044694F84200202801D073
:10226000022038BD71B16AB1012020630020606393
:10227000204600F013FE0346206B012804D0012302
:10228000184638BD012038BD2068016840680090BC
:1022900020680C3050E8001F41F0100140E80012A7
:1022A000002AF5D1ECE7000030B50F4D026800239D
:1022B0000124AA4205D10D4AA2F80018535482F80D
:1022C000024800680A4A90420CD10A48A0F8001857
:1022D000D214914201D9A0F80028B0F80018435454
:1022E00080F8024830BD000000440040FC0100209E
:1022F00000480040000A002010B5044620684069EC
:10230000C0F3C01094F84110212911D180B1206888
:10231000143050E8001F21F0800140E80012002A2C
:10232000F5D1A06B08B1FEF745FA204600F043FD59
:1023300020684069C0F3801094F84210222911D11E
:1023400080B12068143050E8001F21F0400140E8BF
:102350000012002AF5D1E06B08B1FEF72BFA2046F7
:1023600000F0F5FC002010BD70470000F8B50446F1
:1023700022681068D168536900F00F06002E08D15A
:10238000850606D58D0604D52046BDE8F84000F048
:1023900020BD0025002E66D003F0010601F49077E1
:1023A000374360D0C20705D0CA0503D5626C42F03E
:1023B00001026264420705D5DA0703D0626C42F07D
:1023C00002026264820705D5DA0703D0626C42F02C
:1023D00004026264020707D501F02002324303D0F1
:1023E000626C42F008026264626C002A31D080069E
:1023F00004D5880602D5204600F0EBFC2068406931
:10240000C0F38010616C090700D438B3204600F097
:102410009EFC2068406940061CD52068143050E8B6
:10242000001F21F0400140E80012002AF5D1E06BC6
:1024300060B159494163E06BFEF7E0F9002808D02C
:10244000E06B416B01B0BDE8F04008472046FFF764
:102450008BFFF8BD2046FFF787FFF8BD2046FFF74A
:1024600083FF6564F8BD236B012B7DD1C3067BD54B
:10247000CB067ED510685068009050694FF020035D
:1024800040064FF0020643D5E16B0868406880B211
:102490000028E7D0A28D8242E4D9E085886920280F
:1024A0002DD020680C3050E8001F21F4807140E8E6
:1024B0000012002AF5D12068143050E8001F21F0E6
:1024C000010140E80012002AF5D12068143050E8DC
:1024D000001F21F0400140E80012002AF5D184F8E5
:1024E0004230256320680C3050E8001F21F01001B5
:1024F00040E80012002AF5D1E06BFEF75BF9666355
:10250000A08DE18D401A81B22046FFF7CDFEF8BDC7
:10251000A08DE18D401A81B2E08D0028F7D000290E
:10252000F5D020680C3050E8002F22F4907240E87B
:102530000027002FF5D12068143050E8002F22F03A
:10254000010240E80027002FF5D184F842302563CE
:1025500020680C3050E8002F22F0100240E80023E1
:10256000002BF5D1666300E003E02046FFF79CFEF8
:10257000F8BD020606D50A0604D52046BDE8F84097
:1025800000F0D6BC4006F3D54806F1D52046BDE89C
:10259000F84000F003BC0000512C000810B50446C0
:1025A000174A20681749904212D1C86920F40030B8
:1025B000C8610F211448FEF755FBE06BFEF76AF97E
:1025C000A06BFEF767F9BDE810402620FEF720BD9E
:1025D0000E4A904213D1C86920F48020C8614FF49C
:1025E00040610B48FEF73EFBE06BFEF753F9A06B32
:1025F000FEF750F9BDE810402720FEF709BD10BDD9
:102600000044004000100240000801400048004023
:10261000000C014070477047084B0168084A994216
:1026200003D111025160FFF767BE064B994203D1F7
:1026300020215160FFF760BE704700000044004059
:102640000000024000480040FEE7F0B500230A25E4
:1026500030263727002412E0B5EB107F04D906EBB3
:10266000107C01F813C003E007EB107C01F813C0E5
:10267000000101EB430C8CF801405B1CDBB2934280
:10268000EAD3F0BD08B51548416941F00101416147
:10269000406900F001000090002211460C20FEF776
:1026A000D5FC0C20FEF7C5FC002211460D20FEF7DC
:1026B000CDFC0D20FEF7BDFC002211461020FEF7D8
:1026C000C5FC1020FEF7B5FC002211461120FEF7D4
:1026D000BDFCBDE808401120FEF7ABBC0010024075
:1026E00010B586B00020049005901E48816941F025
:1026F00010018161816901F010010191816941F04E
:1027000020018161816901F020010191816941F01D
:1027100004018161816901F004010191816941F045
:1027200008018161806900F0080001904FF4604069
:1027300002900324039402A90B48FEF709FB48F218
:10274000F0700290039402A90848FEF701FB4FF2D3
:10275000FF300290039402A90548FEF7F9FA06B08B
:1027600010BD0000001002400010014000080140B0
:10277000000C014010B501F097FD00220F491048F0
:1027800001F005F808B1FDF7ACFE0E490C4801F068
:10279000FBF908B1FDF7A5FE0B49094800F014FD4F
:1027A00008B1FDF79EFE064801F0A0FA002803D00C
:1027B000BDE81040FDF795BE10BD000038000020B8
:1027C000A4130020C401002094000020FEE7FEE7CF
:1027D0002DE9F05F04464FF006084FF002094FF470
:1027E0008067D8E1B0F8441001F00F06F6B330F876
:1027F00026A05FEA0A417DD530F8261040F68F7298
:10280000114041F0800120F8261006EB860004EB11
:10281000C00505F5A875287B00286CD0E87802284B
:102820006AD02978206830F8212048F68F731A4042
:1028300048F2C0031A4320F821202978206830F894
:10284000212052047ED5B0F8502009EBC10111447B
:1028500007EB4101415AC1F3090BBBF1000F04D052
:102860002A895B46696902F068F9EAE0FFE7C90670
:102870002BD4018848F60F72114041F400410180C9
:1028800004F110052068B0F850102A7809EBC20254
:10289000114407EB4101405AC0F30900E86169693E
:1028A0000844686100212046FEF733FC607B002865
:1028B00097D0A869002894D1607B216840F08000FF
:1028C000A1F84C000020607365E104F5A87501884B
:1028D0000A0521D5B0F850102A7808EBC20211443D
:1028E00007EB4101405AC0F30903EB61EA8804F5A4
:1028F000267102E0B9E076E08AE0206802F01DF976
:102900002068018840F68F72114041F080010180FB
:102910002046FFF7B5F83EE10904D5D5018840F619
:102920008F72114041F0800101802068B0F8501092
:102930002A7808EBC202114407EB4101405AC0F368
:10294000090000E06BE0E86170B1696961B183B2D0
:10295000EA88206802F0F1F8E9696869084468616A
:1029600000212046FEF7DEFB206801880A05ABD473
:10297000C1F301310329A7D0B0F85010084400F288
:102980000C400188C1F30901018029693E290BD956
:102990004A09C90600D1521E01884FF4004343EA98
:1029A0008222114301800BE0C1B14A08C90700D05F
:1029B000521C01884FF6FF7303EA82221143018003
:1029C000206801884BF68F72114081F4805181F4A8
:1029D000005148F2800211430180DCE0018841F49B
:1029E00000410180ECE72068B0F850102A7808EB2D
:1029F000C202114407EB4101415AC1F3090BBBF17B
:102A0000000F1ED0EA885B46696902F096F818E06C
:102A1000524629462046FEF7F5FB834611E0B0F802
:102A2000502008EBC101114407EB4101415AC1F3A9
:102A3000090BBBF1000F04D06A895B46696902F09B
:102A40007CF8E8695844E861686958446861A86995
:102A500010B12869584504D929782046FEF762FB51
:102A600003E02946206801F06BFD5FEA0A6079D532
:102A700006EB860004EBC0011031206830F82620F8
:102A800048F60F731A4042F4004220F82620C87816
:102A9000012814D05FEACA5079D42068B0F85020D9
:102AA0000B7809EBC3031A4407EB4202805AC0F3C8
:102AB00009008A69824256D9121A8A6155E00023B8
:102AC0008B61087B30B35FEA4A6024D5487810B147
:102AD000012814D042E02068B0F8502010440A7851
:102AE00009EBC20200EB420000F580600288C2F3ED
:102AF00009020280028842F4004202802EE020682F
:102B0000B0F8502010440A7809EBC20200EB4200F2
:102B1000A0F8003422E020684A7812B1012A13D0CC
:102B20001CE0B0F8502010440A7808EBC20200EB19
:102B3000420000F580600288C2F309020280028828
:102B400042F40042028009E0B0F8502010440A78B4
:102B500008EBC20200EB4200A0F8003409782046DE
:102B6000FEF7D7FA17E000228A618A6952B14A69F2
:102B700002444A61CA691044C861206801F0E0FC5F
:102B800009E004E009782046FEF7C3FA03E0524664
:102B90002046FEF7B3FB2068B0F8441009043FF567
:102BA00021AE0020BDE8F09F7047000008B507493E
:102BB0004FF4FA520968B1FBF2F14143009100BFB2
:102BC0000098411E0091FAD208BD0000E4000020E8
:102BD0007047FEF7C3B930B593B0282109A8FDF7B7
:102BE00048FB142104A8FDF744FB00240094019441
:102BF000029403940121099108040A900B940D9109
:102C00000225109511904FF4E010129009A8FFF7DB
:102C10004BF908B1FDF765FC0F200490059506946B
:102C20004FF4806007900894022104A8FEF7FAFF91
:102C300008B1FDF756FC1020009003946846FEF79B
:102C40006BFF002801D0FDF74CFC13B030BD70477E
:102C500010B5406A0021C185C184FFF785FB10BD16
:102C600070B5446A20684069C0F3C01094F8411000
:102C70000025212904D118B1E584204600F09BF8F5
:102C800020684069C0F3801094F84210222904D1D2
:102C900018B1E585204600F05AF8606C40F010004D
:102CA00060642046FFF760FB70BD10B50146486ABE
:102CB000096809684FF0000389062ED4C3850168AE
:102CC0000C3151E8002F22F4807241E80024002CDE
:102CD000F5D10168143151E8002F22F0010241E8DA
:102CE0000024002CF5D10168143151E8002F22F0A6
:102CF000400241E80024002CF5D1202180F8421048
:102D0000016B012909D101680C3151E8002F22F033
:102D1000100241E80024002CF5D14363016B012926
:102D200002D0FFF777FC10BD818DFFF7BDFA10BD13
:102D300010B5406A01214163016B012902D0FFF700
:102D40006AFC10BD818D4908FFF7AEFA10BD01681D
:102D50000C3151E8002F22F4907241E80023002B3F
:102D6000F5D10168143151E8002F22F0010241E849
:102D70000023002BF5D1016B012909D101680C3129
:102D800051E8002F22F0100241E80023002BF5D17A
:102D9000202180F8421000210163704710B50168BE
:102DA000CA6822F04002CA60202180F84110FFF773
:102DB00033FC002010BD01680C3151E8002F22F0D7
:102DC000C00241E80023002BF5D1202180F84110FA
:102DD000704708B590F84210222901D0022008BDA2
:102DE00082684FF480539A4201D1016921B1816A0E
:102DF0009A421DD052B10BE0816A02685268C2F358
:102E000008020A80816A891C816209E002697AB13C
:102E10000268526802F07F020A70816A491C81626E
:102E2000C18D491E0904090CC18505D0002008BDCB
:102E3000026852680A70F0E70168CA6822F020024E
:102E4000CA600168CA6822F48072CA6001684A696F
:102E500022F001024A61202180F8421000214163E2
:102E6000026B012A03D0FFF7D5FB002008BD0163E8
:102E700001680C3151E8002F22F0100241E80023D4
:102E8000002BF5D101680A68D20602D50A684968A4
:102E90000091818DFFF708FAE7E7000037B582B0AF
:102EA00004461346039AA262A3850020606422218F
:102EB00084F84210E56B1B49A962E56B1A49E96287
:102EC000E56B1A492963E16B48632168E06B091DD2
:102ED000FDF7C4FD2068016840680190206948B191
:102EE00020680C3050E8001F41F4807140E8001267
:102EF000002AF5D12068143050E8001F41F001018C
:102F000040E80012002AF5D12068143050E8001F74
:102F100041F0400140E80012002AF5D105B0002040
:102F200030BD0000AB2C0008312D0008612C0008DA
:102F300090F84110212901D0022070478168B1F535
:102F4000805F01D1016961B1016A4A1C02620268B5
:102F500009785160C18C491E0904090CC1840AD04A
:102F600013E0016A02680988C1F308015160016A2F
:102F7000891C0162EEE70168CA6822F08002CA601B
:102F80000068C16841F04001C16000207047000046
:102F900010B50548FFF7EAF9BDE810404FF40062AC
:102FA00002490148FFF756B904120020FC01002035
:102FB00010B50548FFF7DAF9BDE810404FF400629C
:102FC00002490148FFF746B94C120020000A0020D0
:102FD0002DE9F041D0F8B822D0F8C062002A19D00B
:102FE00001EB810400EB84030027DD693DB106EBB2
:102FF000C404246AB5FBF4F604FB165424B1C2F8E9
:1030000014720020BDE8F081DF6100231A4600F051
:103010009EFDF6E70220F5E770B50546D5F8B84203
:10302000284600F093FCC4F80C02D5F8B80248B169
:10303000D5F8BC12D4F80402CA6804F503719047AD
:10304000002070BD022070BD70B5044600268121AD
:10305000204600F0BBFB0025E5620121204600F080
:10306000B5FBC4F86C518221204600F0AFFB25640B
:10307000D4F8B80240B104F52E7460684068804707
:10308000206800F094FF2560304670BD10B5D0F880
:10309000B842D0F8BC1200290BD094F80002FF28E7
:1030A00007D08B6894F8012221469847FF2084F8C6
:1030B0000002002010BD00000A2101800048704776
:1030C000EC00002043210180004870473C010020B3
:1030D0004321018000487047F8000020432101800F
:1030E00000487047800100202DE9F0410446002689
:1030F000207C01254FF40077002832D040230222A3
:103100008121204600F073FCE56240230222012168
:10311000204600F06CFCC4F86C5108230322822185
:10312000204600F064FC25644FF4077000F040FF77
:10313000C4F8B80228B30546D4F8BC02006880473A
:103140000020C5F81402C5F81802207CD8B140232D
:1031500001212046D5F8042200F055FC3046BDE898
:10316000F0813B4602228121204600F040FCE562CE
:103170003B4602220121204600F039FCC4F86C5184
:10318000CBE70126EAE73B4601212046D5F8042299
:1031900000F039FCE2E710B5D0F8B812002911D0E0
:1031A000027C3AB1D1F804224023012100F02BFC2B
:1031B000002010BDD1F804224FF40073012100F06B
:1031C00022FCF5E7022010BD02460220002902D0B1
:1031D000C2F8BC1200207047D0F8B802C0F8041240
:1031E00000207047D0F8B802C0F80812C0F81022CA
:1031F000002070472DE9FC4105460C46D5F8B87211
:103200000020019000900026207810F060012DD061
:10321000202907D02146284600F0A2F80226304691
:10322000BDE8FC81E288CAB100060BD5D5F8BC1216
:1032300060788B6839469847E2883946284600F01E
:10324000B5F8ECE7607887F80002A07987F801020A
:10325000E2883946284600F08FF8E0E7D5F8BC123E
:10326000607800228B6821469847D8E7607848B19B
:103270000A2817D00B2825D02146284600F070F8E0
:103280000226CCE795F89C02032805D02146284663
:1032900000F066F80226C2E702226946284600F0DE
:1032A00085F8BCE795F89C02032805D021462846FE
:1032B00000F056F80226B2E7012201A9284600F0E4
:1032C00075F8ACE795F89C020328A8D0214628465B
:1032D00000F046F80226A2E710B5D0F8B81200298F
:1032E00012D0D1F814220AB1012010BD01F50271EB
:1032F0000122CA608A6802630A8993B20A6881213E
:1033000000F025FC002010BD022010BD10B5D0F843
:10331000B42252689047002010BD90F89C22012AE8
:1033200005D0022A03D0032A01D000F019B8498839
:10333000012904D10021C0F8A41200F044B870475C
:1033400010B513460A46002100F05DFB002010BDB9
:1033500010B513460A46002100F0F9FB002010BD0D
:1033600010B504468021204600F0CEFB2046BDE883
:103370001040002100F0C8BB10B50323C0F8943200
:10338000C0F85C21C0F8602113460A46002100F015
:103390003AFB002010BD10B50521C0F8941200239F
:1033A0001A46194600F02FFB002010BD10B502236D
:1033B000C0F89432C261026213460A46002100F04E
:1033C000C6FB002010BD10B50421C0F894120023E4
:1033D0001A46194600F0BBFB002010BD10B504468C
:1033E000012084F89C02D4F8B40221794268204676
:1033F0009047204600F09AFB204600F09EFA0020FD
:1034000010BD000010B5002806D00A46054906A0E8
:1034100000F08CF9034810BD0A46024902A000F0F2
:1034200085F9F7E7601B002043444320436F6E6635
:10343000696700001220088000487047580000208B
:1034400010B5002806D00A46054906A000F06EF91E
:10345000034810BD0A46024902A000F067F9F7E7E9
:10346000601B002043444320496E746572666163AB
:1034700065000000042008800048704754000020C8
:1034800010B50A46024903A000F050F9004810BDEB
:10349000601B002053544D6963726F656C656374E3
:1034A000726F6E696373000010B5002806D00A467B
:1034B000054906A000F03AF9034810BD0A46024942
:1034C00002A000F033F9F7E7601B002053544D339E
:1034D00032205669727475616C20436F6D506F7243
:1034E0007400000010B51A200880FDF747F9014864
:1034F00010BD00006C0000200A46D188012902D0CE
:103500001146FFF72DBF90F89C12012906D0022921
:1035100004D0032909D01146FFF722BF00218160A2
:10352000012200F10801FFF741BF0122011DFFF751
:103530003DBF2DE9F84304460F46002000900026C9
:1035400000257888010A082970D2DFE801F0AB0471
:103550000C22ABAB8B9AD4F8B012207C0A68694677
:1035600090470646A3E0207C4FF0020840B1D4F813
:10357000B402C16A68468847064686F8018096E02C
:10358000D4F8B402816A68468847064686F8018006
:103590008DE0C0B206285FD2DFE800F003122130D0
:1035A0003F4FD4F8B002426822B1207C6946904770
:1035B00006467CE039462046FFF7D2FE012576E03C
:1035C000D4F8B002826822B1207C69469047064652
:1035D0006DE039462046FFF7C3FE012567E0D4F8C9
:1035E000B002C26822B1207C6946904706465EE080
:1035F00039462046FFF7B4FE012558E0D4F8B00262
:10360000026922B1207C6946904706464FE0394660
:103610002046FFF7A5FE012549E0D4F8B002426933
:103620002AB1207C69469047064640E03AE0394698
:103630002046FFF795FE012539E0D4F8B0028269F3
:1036400022B1207C69469047064630E03946204644
:10365000FFF786FE01252AE039462046FFF780FE67
:10366000012524E0207C28B139462046FFF778FE6A
:1036700001251CE0D4F8B402416B68468847064631
:1036800015E0207C28B139462046FFF769FE012568
:103690000DE0D4F8B402016B68468847064607215E
:1036A000717004E039462046FFF75AFE0125002DCF
:1036B00012D1BDF8000048B1FA883AB1824200D96F
:1036C0000246009231462046FFF770FEF888002837
:1036D00002D12046FFF777FEBDE8F883002102E023
:1036E000491CC9B2401C0278002AF9D1084670472B
:1036F0000A4690F89C12012906D0022904D0032919
:1037000002D01146FFF72CBED188022902D0114603
:10371000FFF726BE0121C160D0F8A41209B1032130
:10372000C160022200F10C01FFF740BE70B50446F3
:103730000D461646002C17D02046FFF7CFFF02217A
:1037400001EB40003080307828700321022069703E
:10375000002306E0411CC9B22A54641C481CC0B2B4
:103760006B542278002AF5D170BD01460020002953
:1037700006D0012905D0022905D0032905D0022051
:10378000704702207047012070470220704710B533
:10379000002810D0D0F8B43213B10023C0F8B432EE
:1037A00009B1C0F8B012012180F89C12027000F03B
:1037B000D1F8002010BD022010BD10B5D0F8C00215
:1037C000FDF7F4FCBDE81040FFF7CFBF10B5D0F80F
:1037D000C002FDF7C7FCBDE81040FFF7C6BF70B5DB
:1037E00004461346002909D0D4F8B40242691AB13C
:1037F00094F89C02032859D0022070BD04F11400F3
:10380000D4F894120025022903D0042940D0F1B342
:1038100042E0D0E903218A420DD9511AC1608AB22F
:1038200019462046FFF794FD00231A461946204604
:1038300000F0E9F830E08068B0FBF1F201FB120221
:103840009AB9884211D3D4F8981288420DD2002236
:1038500011462046FFF77CFDC4F8985200231A4613
:103860001946204600F0CFF816E0D4F8B402C1683B
:1038700029B194F89C02032801D120468847802171
:10388000204600F041F92046FFF785FD04E0FFE700
:103890008021204600F038F994F8A002012807D1D1
:1038A000204600F07AF984F8A05201E020469047C3
:1038B000002070BD70B5044608461146002809D0A6
:1038C000D4F8B4128A691AB194F89C1203292FD043
:1038D000022070BD04F5AA70D4F89432032B02D0F4
:1038E000052B1DD027E0D0E903539D420AD9EB1ADE
:1038F000C3600069834200D303469AB22046FFF7B3
:103900001FFD18E0D4F8B402016929B194F89C02B3
:10391000032801D1204688472046FFF754FD0AE0DE
:103920000020C4F894020021204600F0EDF802E0E7
:10393000014620469047002070BD10B5D0F8C00267
:10394000FDF7FAFBBDE81040FFF70FBFD0F8C0024B
:10395000FDF79FBE10B504461B48C0F8D442C4F81A
:10396000C0021A4901600821017102218171002100
:103970008172C1720173FDF7C2FF08B1FCF7B1FD9E
:1039800004F530740022182311462068FDF7A2FBCD
:103990005823002280212068FDF79CFBC0230022D1
:1039A00081212068FDF796FB4FF4887300220121E6
:1039B0002068FDF78FFB4FF480730022822120687E
:1039C000FDF788FB002010BD88180020005C004037
:1039D0000A0601F07F01D0F8C00201EB810100EB83
:1039E000C10001D5807C704790F85201704710B536
:1039F00014461A46D0F8C0022346FDF753FEBDE830
:103A00001040FFF7B2BE10B5D0F8C002FDF775FE4A
:103A1000BDE81040FFF7A9BE70B504460022402360
:103A200011462046FFF7E3FF0125C4F85851402610
:103A3000C4F864614023002280212046FFF7D7FFAD
:103A4000A561666284F89C520020C4F8940260600C
:103A5000C4F8A402D4F8B80228B1D4F8B402002102
:103A6000426820469047002070BD90F89C120429BF
:103A700003D190F89D1280F89C120020704710B579
:103A800090F89C12032904D1D0F8B412C96901B18D
:103A90008847002010BD01740020704710B5D0F891
:103AA000C002FDF7DAFFBDE81040FFF75EBE70B55B
:103AB000044604F52A70054600F052F80120C4F8C7
:103AC0009402B4F8AE02C4F8980294F8A82212F056
:103AD0001F000AD001280DD0022810D002F080016A
:103AE000204600F011F8002070BD2946204600F065
:103AF00002F9F8E72946204600F024FAF3E72946C0
:103B0000204600F02DF9EEE710B5D0F8C002FDF721
:103B100008FEBDE81040FFF728BE10B5D0F8C0027F
:103B2000FDF7B5FFBDE81040FFF71FBE10B5D0F898
:103B3000C002FDF7C5FFBDE81040FFF716BE00F557
:103B4000277001784170042101700020704710B582
:103B5000D0F8C002FDF71CFEBDE81040FFF705BE1F
:103B60000A7802704A7842708A78CB7802EB032296
:103B700042800A794B7902EB032282808A79C979E3
:103B800002EB0121C180704702460020002902D0CB
:103B9000C2F8B4127047022070470020704770B519
:103BA00004468888002821D1C888F8B94888802828
:103BB0001CD200F07F0594F89C0203280DD084F8F5
:103BC0009E5229462046FFF769FF2046FFF7FBFB80
:103BD00045B1022084F89C0270BD2046BDE87040CB
:103BE000FFF7BEBB012084F89C0270BD2046BDE8F3
:103BF0007040FFF7B5BB10B50224D0F8B422002AFC
:103C000003D01268904700B90024204610BD000080
:103C100070B504460E46304DB1782970012905D99A
:103C200031462046BDE87040FFF79ABB94F89C02ED
:103C300002280BD0032823D031462046FFF790FB03
:103C400029782046BDE87040FFF760BB99B16160FC
:103C5000032084F89C022046FFF7CDFF022804D001
:103C60002046BDE87040FFF7AEBB31462046BDE8B8
:103C70007040FFF775BB2046BDE87040FFF7A3BB5F
:103C800091B16068884221D0C1B22046FFF73EFB67
:103C9000297861602046FFF7AEFF022810D0204649
:103CA000BDE87040FFF78FBB022084F89C02616082
:103CB0002046FFF72BFB2046BDE87040FFF783BB93
:103CC00031462046BDE87040FFF74ABB2046BDE8BC
:103CD0007040FFF778BB0000E80000204988012908
:103CE00003D1C0F8A412FFF76EBB704710B5FFF701
:103CF00014FF002010BD10B500240A7812F06002F5
:103D00000CD0202A05D0402A03D0FFF729FB2046FB
:103D100010BDD0F8B42292689047F8E74A780A2A92
:103D20001BD2DFE802F011171A141A08051A0E0B3D
:103D3000FFF7FFFBEBE7FFF732FFE8E7FFF768FF6E
:103D4000E5E7FFF7D9FBE2E7FFF7D2FCDFE7FFF794
:103D5000C5FFDCE7FFF7E1FAD9E7FFF701FBD6E79C
:103D60002DE9F04104460A4600261179137813F034
:103D7000600011D0202808D0402806D011462046E7
:103D8000FFF7EEFA3046BDE8F081D4F8B4021146F0
:103D9000836820469847F5E7C3F3411001280BD00C
:103DA0005078002860D0012837D003280CD0114665
:103DB0002046FFF7D5FAE5E7D4F8B4021146836848
:103DC0002046BDE8F041184794F89C02022806D02E
:103DD000032814D011462046FFF7C2FAD2E749B1B2
:103DE000802907D02046FFF78FFE80212046FFF76D
:103DF0008BFEC7E711462046FFF7B2FAC2E75088AC
:103E000038B931B1802904D0D08810B92046FFF7E5
:103E10007BFE2046FFF7D7FAB4E794F89C0202280D
:103E200006D0032814D011462046FFF799FAA9E7D7
:103E300049B1802907D02046FFF766FE8021204641
:103E4000FFF762FE9EE711462046FFF789FA99E7E1
:103E50005088002896D1480602D02046FFF7ADFCD6
:103E60002046FFF7B0FA8DE794F89C02002702285D
:103E700006D0032824D011462046FFF771FA81E7C7
:103E800031B1802904D011462046FFF769FA79E75D
:103E9000080607D501F07F0000EB800004EB8001ED
:103EA000143107E001F07F0000EB800004EB80019B
:103EB00001F5AA710F6002222046FFF777FA61E749
:103EC00008060CD501F00F0000EB800004EB800029
:103ED000806968B911462046FFF742FA52E701F0BF
:103EE0000F0000EB800004EB8000D0F8580148B1CF
:103EF00008060CD501F07F0000EB800004EB800584
:103F000014350CE011462046FFF72AFA3AE701F093
:103F10007F0000EB800004EB800505F5AA7541B138
:103F2000802906D02046FFF753FD20B101202860EC
:103F300002E02F6000E02F60022229462046FFF7B2
:103F400035FA1FE770B505460C46207810F0600280
:103F500009D0202A07D0402A05D021462846FFF75D
:103F6000FFF9002070BD95F89C22012A08D0022A92
:103F700006D0032A04D021462846FFF7F1F9F0E7DE
:103F8000207901280ED8D5F8B40221468268284647
:103F90009047E1880029E4D10028E2D12846FFF7C4
:103FA00012FADEE721462846FFF7DAF9D9E770472B
:103FB00000487047681600202DE9F04F00270D7863
:103FC00030F8252048F68F131A40CB78002B7CD090
:103FD000012B78D0022B02D0032B79D0012748F295
:103FE0008004224320F825200A7830F8223048F651
:103FF0008F752B401343234320F822300B7B48F26C
:10400000C00648F6BF724FF0040A4CF280084BF627
:104010008F7CE3B3CB78022B7ED00B7830F82390E3
:1040200048F68F6B09EA0B0949EA040920F8239046
:10403000B0F85030034491F8009003EB0913B1F845
:10404000089029F00109A3F80094B0F85030034417
:1040500091F800900AEBC90903EB4903B1F80A9003
:1040600029F00109A3F800944B78002B6BD00B7852
:1040700030F823905FEA494907D530F8239009EAE0
:10408000050949EA080920F823900B7800E025E0AB
:1040900030F823805FEA486807D530F8238008EAC3
:1040A000050848EA060820F82380CB78012B76D053
:1040B0000B7830F82350154085F02002224320F879
:1040C0002320E3E001E006E002E042F4007286E72C
:1040D00042F4C06283E742F4806280E74B788BB39E
:1040E000B0F85030034491F800C003EB0C13B1F862
:1040F00006C02CF0010CA3F800C40B7830F823C0E4
:104100005FEA4C6C07D530F823C00CEA050C4CEA8A
:10411000060C20F823C000E075E0CB78012B09D015
:10412000097830F82130134083F02002224320F830
:104130002120B3E0097830F821301340234320F8E0
:104140002130ABE000E06AE0B0F8502002440B7888
:104150000AEBC30302EB4302CB8823F00103A2F86E
:104160000034B0F8502002440B78062606EBC30357
:1041700002EB430202F580621388C3F30903138044
:104180000B693E2B0CD95E09DB0600D1761E138825
:104190004FF4004949EA8626334313800CE06EE071
:1041A00013B35E08DB0700D0761C13884FF6FF7947
:1041B00009EA8626334313800A7830F822305B04FC
:1041C00006D530F822302B4043EA080320F822308D
:1041D000097871B130F8212002EA0C0282F4005211
:1041E000224320F8212059E0138843F40043138030
:1041F000E2E7018801EA0C0181F4805181F4005169
:10420000214301804AE00B7830F8239009EA050940
:1042100048F2801B49EA0B0920F8239008E70B7845
:1042200030F823905FEA494907D530F8239009EA2E
:10423000050949EA080920F823900B7830F8238013
:104240005FEA486807D530F8238008EA050848EA9D
:10425000060820F823800B7830F8235005EA0C0577
:1042600085F4805585F40055254320F823500978BE
:1042700030F821301340234320F821300EE00B7832
:1042800030F823501540254320F82350097830F8A2
:10429000212002EA0C02224320F821203846BDE802
:1042A000F08F00207047000070B586B000200290AB
:1042B0000390049005901748816941F004018161E1
:1042C000806900F004000190134D4FF480540022E7
:1042D00021462846FCF734FE029401220392022272
:1042E0000492059202A92846FCF732FD00222146DD
:1042F0002846FCF725FE4FF4FA763046FCF7E8FB3B
:10430000012221462846FCF71BFE3046FCF7E0FB65
:1043100006B070BD00100240000801402DE9F043D6
:1043200091F80C904C780A7848F6BF764BF68F7768
:1043300048F2800548F2C00C4CF2800848F68F73B2
:10434000B9F1000F31D07CB330F82240640406D5B7
:1043500030F822401C4044EA080420F822400A7841
:1043600030F82240640606D530F822401C4044EA6A
:104370000C0420F822400A7830F822401C4044EA1D
:10438000080420F822400A7830F8223033402B43CA
:1043900020F82230097830F821203A402A4320F8CA
:1043A00021200020BDE8F08326E094B130F82240BF
:1043B000640606D530F822401C4044EA0C0420F87C
:1043C0002240097830F8212032402A4320F8212069
:1043D000E7E730F82240640406D530F822401C405C
:1043E00044EA080420F82240097830F821203A40B5
:1043F0002A4320F82120D4E730F82240640406D56F
:1044000030F822401C4044EA080420F822400A7890
:1044100030F82240640606D530F822401C4044EAB9
:104420000C0420F822400A7830F822401C4044EA6C
:104430000C0420F822400A7830F822303B402B430D
:1044400020F82230097830F8212032402A4320F821
:104450002120A6E70020704700207047012120F8A6
:10446000401F00210180818001820020704730F8C8
:10447000401F21F43F410180002070470020704719
:1044800030B50A7B002A3BD14A7848F68F7548F24E
:104490008004DAB10A7830F822305B0607D530F8AC
:1044A00022302B4048F2C0052B4320F82230CA7836
:1044B000012A25D0097830F8212048F6BF731A4028
:1044C00082F02002224320F8212019E00A7830F8F7
:1044D00022305B0407D530F822302B404CF28005A7
:1044E0002B4320F82230097830F821204BF68F73C7
:1044F0001A4082F4805282F40052224320F8212094
:10450000002030BD10B54A78097848F28003002AAF
:104510000AD030F8212048F6BF74224082F0100201
:104520001A4320F8212009E030F821204BF68F743F
:10453000224082F480521A4320F82120002010BD2E
:104540002DE9F04F05460C4606276378217B4FF096
:10455000000B4FF0020848F68F724FF400494FF6F7
:10456000FF7A012B09D0002976D0E078022874D098
:10457000012873D00120BDE8F08FA669206986422A
:1045800000D90646D1B1E178022928D0206A801BE3
:104590002062207835F8201049067DD5B5F85010F6
:1045A000294407EBC00001EB4000A0F800646289D9
:1045B000B3B22846616900F0E8FA6BE1B3B2E28871
:1045C0002846616900F0E1FAB5F8500028442178E6
:1045D00008EBC10100EB4100A0F800645AE1216A38
:1045E00081427DD9207835F82010114048F28012A0
:1045F000114325F82010206A801B2062207835F8AE
:10460000201049066DD5617811B101292CD034E014
:10461000B5F85010294407EBC00001EB400000F54D
:1046200080600188C1F3090101803E2E09D971091A
:10463000F20600D1491E028849EA81210A4302801C
:104640001BE066B17108F20700D0491C02880AEA33
:1046500081210A43028010E02CE15FE1DCE1018866
:1046600041F40041018008E0B5F85020511907EBF2
:10467000C00001EB4000A0F800646289B3B2284694
:10468000616900F082FA6069304460612169206AE2
:10469000884204D9801B00E0EDE0206202E006467B
:1046A000C4F820B0607810B101282DD036E0B5F8FC
:1046B00050002844217808EBC10100EB410000F5CF
:1046C00080600188C1F3090101803E2E0CD9710977
:1046D000F20600D1491E028849EA81210A4301E01D
:1046E000ADE022E0028019E04EB17108F20700D07F
:1046F000491C02880AEA81210A4302800EE00188EF
:1047000041F40041018009E0B5F8500028442178C7
:1047100008EBC10100EB4100A0F800642289B3B2AC
:104720002846616900F031FAB4E0617811B10129DD
:1047300029D031E0B5F85010294408EBC00001EB56
:10474000400000F580600188C1F3090101803E2E20
:1047500009D97109F20600D1491E028849EA81216E
:104760000A43028018E04EB17108F20700D0491CDC
:1047700002880AEA81210A4302800DE0018841F49F
:104780000041018008E0B5F85010294408EBC00052
:1047900001EB4000A0F800642289B3B228466169A9
:1047A00000F0F3F96069304460612169206A884251
:1047B00002D9801B206202E00646C4F820B060786F
:1047C00010B101282AD033E0B5F8500028442178F0
:1047D00007EBC10100EB410000F580600188C1F3E7
:1047E000090101803E2E09D97109F20600D1491E46
:1047F000028849EA81210A43028019E04EB171081A
:10480000F20700D0491C02880AEA81210A4302808B
:104810000EE0018841F40041018009E0B5F8501034
:104820004819217807EBC10100EB4100A0F80064B2
:104830006289B3B22846616900F0A7F92AE02078BE
:1048400035F8202048F68F631A4048F280031A4357
:1048500025F82020B5F850002844227808EBC20241
:1048600000EB42008BB2A0F800342289284661692F
:1048700000F08BF90EE0B5F85010294408EBC000A9
:1048800001EB4000A0F800642289B3B228466169B8
:1048900000F07BF9207835F8201048F6BF721140FF
:1048A00081F0100181F0200148F28002114325F8C7
:1048B00020102EE1A1692069814202D9091AA16163
:1048C00002E00846C4F818B0B5F850102944227820
:1048D00007EBC20201EB420101F580610A88C2F3D5
:1048E00009020A803E2809D94209C00600D1521E99
:1048F000088849EA822210430880FBE048B1420858
:10490000C00700D0521C08880AEA8222104308809F
:10491000F0E0088840F400400880EBE023BBB5F8E5
:1049200050002844217808EBC10100EB410000F55C
:1049300080600188C1F30901018021693E2909D9FC
:104940004B09C90600D15B1E018849EA832319433C
:10495000018009E069B14B08C90700D05B1C0188E0
:104960000AEA832319430180607838B1012830D0E6
:104970003AE0018841F400410180F5E7B5F85000C4
:104980002844217807EBC10100EB410000F580606D
:104990000188C1F30901018021693E2909D94B0928
:1049A000C90600D15B1E018849EA832319430180AF
:1049B0001AE049B14B08C90700D05B1C01880AEA1C
:1049C0008323194301800FE0018841F400410180F5
:1049D0000AE0B5F850104819217807EBC10100EB47
:1049E0004100218AA0F80014E069D0B3217835F89D
:1049F0002100430401D5430605D400F4804300F0B0
:104A00004000034376D135F82100104048F2C0023F
:104A1000104325F821006DE0A1692069814202D987
:104A2000091AA16102E00846C4F818B023BBB5F822
:104A300050102944227808EBC20201EB420101F533
:104A400080610A88C2F309020A803E280AD9420915
:104A5000C30600D1521E0B8849EA822213430B8001
:104A60000AE047E068B14208C30700D0521C0B8837
:104A70000AEA822213430B80617839B101292FD0D1
:104A800038E00A8842F400420A80F5E7B5F8501091
:104A90002944227807EBC20201EB420101F5806153
:104AA0000A88C2F309020A803E2809D94209C006D1
:104AB00000D1521E088849EA82221043088019E07A
:104AC00048B14208C00700D0521C08880AEA822276
:104AD000104308800EE0088840F40040088009E098
:104AE000B5F850205119227807EBC20201EB4201C0
:104AF000A1F80004207835F820104BF68F72114091
:104B000081F4805181F4005148F28002114325F86C
:104B1000201000202FE50021403081804FF43F41DC
:104B200001800020704700000148FCF748BE0000EB
:104B300088180020B0F84400704710B55C0800EBFE
:104B4000420000F58060002C08D030F8042B0A7079
:104B5000120A4A70891C641E002CF6D1DA0701D0B3
:104B60000088087010BD00207047002902D1802104
:104B7000A0F84C1000207047012120F8401F0021B0
:104B80008180032101800020704710B55B1C5B0809
:104B900000EB420000F58060002B09D00A784C78C9
:104BA00042EA042220F8042B891C5B1E002BF5D15D
:104BB00010BDFEE70907090E002804DB00F1E02024
:104BC00080F80014704700F00F0000F1E02080F83A
:104BD000141D7047002211F8013B00F8013B521CE4
:104BE000042AF8DB7047002211F8013B00F8013B72
:104BF000521C022AF8DB70472DE9F041FCF71EF841
:104C0000174940F23510C86020241648006800F2A9
:104C1000FF30C11700EB9150851220354FF4167705
:104C2000202D06D2022000F0A3FA3846FBF750FFF1
:104C3000F8E74FF000660FE006EB84200121FBF758
:104C400052FC40B1FBF7AAFF022000F091FA38466F
:104C5000FBF73EFFF8E7641CAC42EDD9BDE8F081FC
:104C600000200240C400002008B5002080F3108816
:104C7000FCF77CF9FDF7AFFFFCF76AF9BF4C206346
:104C800010B90F20FCF784F9FDF72AFDFDF7FAFCB7
:104C9000FDF770FD4FF41670FBF71AFFB749B84FD8
:104CA0000222091D3846FBF769FCB4F9040041F201
:104CB00001060025B04209D1A580B0490222091D94
:104CC0003846FBF7C9FC6420FBF702FFAD48AE4F46
:104CD000007807F1020918B917E06420FBF7F8FE25
:104CE00001213846FBF7FFFB0028F6D1009602E0D1
:104CF0006420FBF7EDFE022269464846FBF7ACFC58
:104D00000028F5D16420FBF7E3FE9C490222891CB0
:104D10004846FBF733FCB4F90200B04277D10120DA
:104D200000F026FADFF864B2DFF86482DFF86492FC
:104D3000994E1527DFF864A29AF80000012806D0E2
:104D400002282DD0032874D0042873D0C1E09448E1
:104D5000017889B105709348A06093480580934815
:104D600005803770C82088F80000A9F800506561F8
:104D7000A561E561256265628D48007800280ED046
:104D80008BF80050FFF738FF01208BF800006420FB
:104D9000FBF79EFE02208AF800008548057098E027
:104DA000DFF810A29AF80000002818D07E497F484A
:104DB000B1F90010B0F900004A1C904228D17E4899
:104DC0007E4900784208A068FBF788FC40B18AF869
:104DD000005001208BF80000A069401CA06178E021
:104DE0008AF8005001208BF800006F480188491CA8
:104DF0000180E068A0603770C92088F800006B4827
:104E00000088A9F800006069401C606161E076E0FC
:104E1000884210D18AF8005001218BF800103770B9
:104E2000C92188F80010A9F80000E069401CE06181
:104E30004FE00CE049E08AF800503770C92188F84B
:104E40000010A9F80000206A401C206241E05C4884
:104E5000017859B105703770CA2088F800005348AE
:104E60000088A9F80000FCF773F82061FCF770F8DF
:104E70002169401A40F2DC5188422AD9002000F012
:104E800077F9FBF78BFE6420FBF722FEDFF814A115
:104E9000DAF800004FEA8A0188420FD8DAF80000F9
:104EA000B0F1005F0AD3FBF795FADAF80400E0628C
:104EB000A062DAF8001081F3088880476420FBF7CD
:104EC00007FE36480421017003E04FF41670FBF72B
:104ED000FFFD307838B115287FF42CAF00F01EF9B3
:104EE000C820307026E74FF4167A5046FBF7F0FDE5
:104EF0005046FBF7EDFD012000F03AF91AE7294D85
:104F0000286830490840B0F1005F09D1FBF762FA28
:104F100028686868E062A062296881F30888804791
:104F20004FF416784046FBF7D3FD4D464046FBF75D
:104F3000CFFD2078401CC0B220700A28F6D902E0CC
:104F40006420FBF7C5FD01213846FBF7CCFA0028A9
:104F5000F6D1009602E06420FBF7BAFD0222694612
:104F60002846FBF779FB0028F5D1FBF717FEC82090
:104F7000FBF7AEFDFCF79CF8D8E70000000000202E
:104F800002780008A9000020007C0008B000002082
:104F9000A8000020B8000020A4000020AE000020DF
:104FA000AA00002000800008BC000020BA000020F9
:104FB000AB000020AD000020AF00002068250020DD
:104FC000AC0000200000FE2F2DE9F047504C94F873
:104FD0000E9084F80F9094F80DC084F80EC0227BD8
:104FE0006273E37A2373A17AE172A07294F809A044
:104FF0000125484E4FF0000804F12007BAF1000FD8
:1050000060D0A1694A1CA2617054B91D48788978A2
:10501000C0F58572531A7A78934203DA84F80980CE
:10502000C4F8188010440144A06981420BD884F868
:105030000980C4F818803748FBF78AFB28B1364945
:105040000868401C0860BDE8F0877879C8280FD050
:10505000C92815D0CA28F6D1E069FA2190FBF1F0F1
:10506000B4F914108842EEDCA079022826D027E09B
:105070002748B11D1C30FFF7ADFDA571A570E2E713
:10508000A07902280BD00128DDD12148B11D1230B2
:10509000FFF7A9FD608A0128D5D1E570D3E76079D3
:1050A0000028D0D184F8088065711948B11D1230EC
:1050B000FFF799FD7878801EE071C4E70320A071A6
:1050C0002571C0E797F80080C84517D197F803808D
:1050D000984513D197F8048088450FD1657287F8F9
:1050E00001C0BA70787186F8009086F801C0B2707D
:1050F000F370317170710620A061A4E7242AA2D157
:10510000412BA0D149299ED144289CD165709AE7B2
:10511000A8000020602500203400002010B51249AE
:10512000124C0878207060704879A070C878E070E0
:105130000879207115206071A1F126000078A07116
:10514000E01D163900F044F8032060700921204664
:10515000FBF7FEFA6072000AA0722046BDE810401C
:105160000B21FBF721B90000CE0000206C260020A7
:1051700070B50646144D4FF485711448FBF757F887
:1051800005F12601114C0A78012022704A79A2709B
:10519000CA78E27009792171C72161710721E9821A
:1051A000A67160702046FBF7D3FAE98A4A1C92B2D6
:1051B0006054030A501C81B2E982A3542046BDE822
:1051C0007040FBF7F1B80000A80000206C2600201A
:1051D000002211F8013B00F8013B521C022AF8DBC7
:1051E0007047010202030405060708090A0B0C0DAB
:1051F0000E0F101000000000000000000102030468
:105200000607080900C1814001C0804101C08041FA
:1052100000C1814001C0804100C1814000C1814086
:1052200001C0804101C0804100C1814000C1814076
:1052300001C0804100C1814001C0804101C0804166
:1052400000C1814001C0804100C1814000C1814056
:1052500001C0804100C1814001C0804101C0804146
:1052600000C1814000C1814001C0804101C0804136
:1052700000C1814001C0804100C1814000C1814026
:1052800001C0804101C0804100C1814000C1814016
:1052900001C0804100C1814001C0804101C0804106
:1052A00000C1814000C1814001C0804101C08041F6
:1052B00000C1814001C0804100C1814000C18140E6
:1052C00001C0804100C1814001C0804101C08041D6
:1052D00000C1814001C0804100C1814000C18140C6
:1052E00001C0804101C0804100C1814000C18140B6
:1052F00001C0804100C1814001C0804101C08041A6
:1053000000C1814000C0C101C30302C2C60607C775
:1053100005C5C404CC0C0DCD0FCFCE0E0ACACB0BE5
:10532000C90908C8D81819D91BDBDA1A1EDEDF1F15
:10533000DD1D1CDC14D4D515D71716D6D21213D305
:1053400011D1D010F03031F133F3F23236F6F737B5
:10535000F53534F43CFCFD3DFF3F3EFEFA3A3BFBA5
:1053600039F9F83828E8E929EB2B2AEAEE2E2FEF55
:105370002DEDEC2CE42425E527E7E62622E2E323C5
:10538000E12120E0A06061A163A3A26266A6A767F5
:10539000A56564A46CACAD6DAF6F6EAEAA6A6BAB65
:1053A00069A9A86878B8B979BB7B7ABABE7E7FBF95
:1053B0007DBDBC7CB47475B577B7B67672B2B37385
:1053C000B17170B050909151935352929656579735
:1053D000559594549C5C5D9D5F9F9E5E5A9A9B5B25
:1053E00099595898884849894B8B8A4A4E8E8F4FD5
:1053F0008D4D4C8C44848545874746868242438345
:10540000418180402454000800000020FC0100007D
:1054100028010008F4540008FC010020FC3C0000B6
:1054200084010008911280022C081335341B087582
:10543000041A81041AA9041AE5041A05041A41047D
:1054400017040309041201140202021640830440E7
:105450005726020102030103261A031349031B08FE
:1054600045041A3D041A6D04C11947011532FE1294
:10547000059CFE060228821053127A130A06291F81
:105480002A401C1C09024397111DC03209042D1A21
:10549000020B130524161001052401100901042430
:1054A0000202052406170107058203081C100904DF
:1054B000CD320A1D07050102432C07058107093873
:1054C000442A40072A8107112B0907440A3B044458
:1054D00013E9301B08490413F53142081A8D0C13E7
:1054E000D12F1B081908C11AD1101AC5041ADD04DE
:0454F0001AB90400E1
:04000005080000ED02
:00000001FF
